:020000040800F2
:1000000000000320613700084F080008510800086D
:1000100053080008550800085708000800000000B1
:10002000000000000000000000000000312D00086A
:100030005908000800000000D12D00085B080008E6
:10004000B1370008B1370008B1370008B1370008F0
:10005000B1370008B1370008B1370008B1370008E0
:10006000B1370008B1370008B1370008B1370008D0
:10007000B1370008B1370008B1370008B1370008C0
:10008000B1370008B1370008B1370008B1370008B0
:10009000B1370008B1370008B1370008B1370008A0
:1000A000B137000865080008B1370008B13700080B
:1000B000B1370008B1370008B1370008B137000880
:1000C000B1370008B1370008B1370008B137000870
:1000D000B1370008B1370008B1370008B137000860
:1000E000B1370008B1370008B1370008B137000850
:1000F000B1370008B1370008B1370008B137000840
:10010000B1370008B1370008B1370008B13700082F
:10011000B1370008B1370008B1370008B13700081F
:10012000B1370008B1370008B1370008B13700080F
:10013000B1370008B1370008B1370008B1370008FF
:10014000B1370008B1370008B1370008B1370008EF
:10015000B1370008B1370008B1370008B1370008DF
:10016000B1370008B1370008B1370008B1370008CF
:10017000B1370008B1370008B137000800000000AF
:10018000B1370008B1370008B1370008B1370008AF
:10019000B1370008B1370008B1370008B13700089F
:0C01A000B1370008B1370008B137000883
:1001B00010B5054C237833B9044B13B10448AFF3A1
:1001C00000800123237010BD0C00002000000000FF
:1001D000FC37000808B5034B1BB103490348AFF3D4
:1001E000008008BD0000000010000020FC3700085F
:1001F00053B94AB9002908BF00281CBF4FF0FF318E
:100200004FF0FF3000F072B9ADF1080C6DE904CE8B
:1002100000F006F8DDF804E0DDE9022304B07047E1
:100220002DE9F047089E04468846002B4BD18A42B0
:10023000154667D9B2FA82F24AB1C2F1200701FA33
:1002400002F320FA07F7954047EA030894404FEA83
:10025000154E230CB8FBFEF71FFA85FC0EFB178822
:1002600043EA084307FB0CF1994209D9EB1807F15F
:10027000FF3080F01B81994240F21881023F2B44ED
:100280005B1AA4B2B3FBFEF00EFB103344EA034446
:1002900000FB0CFCA44509D92C1900F1FF3380F0B8
:1002A0000781A44540F2048102382C4440EA07400B
:1002B000A4EB0C0400271EB1D4400023C6E9004380
:1002C0003946BDE8F0878B4209D9002E00F0EB805B
:1002D0000027C6E9000138463946BDE8F087B3FA81
:1002E00083F7002F47D18B4202D3824200F2FA807B
:1002F000841A61EB030301209846002EE0D0C6E982
:100300000048DDE702B9FFDEB2FA82F2002A40F0CF
:100310008F80491B4FEA154E1FFA85F80127B1FB64
:10032000FEFC230C0EFB1C1143EA014308FB0CF1FD
:10033000994207D9EB180CF1FF3002D2994200F232
:10034000CD808446591AA3B2B1FBFEF00EFB101407
:1003500043EA044408FB00F8A04507D92C1900F132
:10036000FF3302D2A04500F2B6801846A4EB080481
:1003700040EA0C409FE7C7F1200CBB4022FA0CFE7C
:100380004EEA030E01FA07F420FA0CF521FA0CF3F9
:100390004FEA1E482543B3FBF8F92C0C08FB193330
:1003A0001FFA8EFA44EA034309FB0AF49C4202FA5C
:1003B00007F200FA07F10BD91EEB030309F1FF3036
:1003C00080F087809C4240F28480A9F10209734446
:1003D0001B1BADB2B3FBF8F008FB103345EA034436
:1003E00000FB0AFAA24508D91EEB040400F1FF3312
:1003F0006BD2A24569D90238744440EA0940A0FB97
:100400000289A4EB0A044C45C2464B4654D351D052
:10041000002E69D0B1EB0A0564EB030404FA0CFC6E
:10042000FD40FC404CEA0505C6E90054002747E7BB
:10043000C2F1200320FA03F7954001FA02F021FAF5
:1004400003F34FEA154E3843010CB3FBFEF71FFAD6
:1004500085F80EFB173341EA034107FB08F38B4293
:1004600004FA02F407D9691807F1FF3C2FD28B4236
:100470002DD9023F2944CB1A81B2B3FBFEF00EFB0B
:10048000103341EA034100FB08F38B4207D9691896
:1004900000F1FF3C17D28B4215D902382944C91A02
:1004A00040EA07473BE73746304609E70746E7E6B5
:1004B0001846FBE64145ABD2B8EB020A69EB0E02E7
:1004C00001381346A4E76046E9E7184695E7674612
:1004D000D1E781467CE702382C4447E7ACF1020CB7
:1004E0002B442FE7384608E73746E9E6704700BF58
:1004F0002DE9F0418CB000240194424B1A6B42F07C
:1005000004021A631A6B02F004020192019A029427
:100510001A6B42F080021A631A6B02F08002029298
:10052000029A03941A6B42F001021A631A6B02F0EA
:1005300001020392039A04941A6B42F002021A63B6
:100540001A6B02F002020492049A05941A6B42F0AC
:1005500008021A631A6B02F008020592059A0694C3
:100560001A6B42F040021A631B6B03F040030693C0
:10057000069BDFF8A08022464FF48141404602F0FE
:1005800041F9214F22464021384602F03BF91F4DE8
:1005900022464FF40071284602F034F94FF400531C
:1005A00007931B4B0893099407A9284601F094FF71
:1005B0004FF4814307930126089609940A9407A9EA
:1005C000404601F089FF40230793089609940A9456
:1005D00007A9384601F080FF802307930894099407
:1005E00007A9384601F078FF4FF400730793089687
:1005F00009940A9407A9284601F06EFF0CB0BDE8E3
:10060000F08100BF0038024000180240000802409C
:10061000000011100004024008B50B4C00224FF4FA
:100620008141204602F0EEF84FF4967003F087F80F
:1006300001224FF48141204602F0E4F84FF4967015
:1006400003F07DF8E9E700BF0004024008B5026846
:10065000034B9A4200D008BD02F0B8F9FBE700BF97
:1006600000000140FEE7000000B583B01248134BC4
:10067000036001234360002303828DF80030802251
:100680008DF80120E1228DF802208DF803308DF8DD
:1006900004308DF80530C0F814D08361C3614FF485
:1006A0000003036200F076FB10B903B05DF804FBB1
:1006B000FD210348FFF7D6FFA8410020008002403B
:1006C0002838000808B50B480B4B03604FF4E133A2
:1006D000436000238360C36003610C224261836135
:1006E000C36101F079F800B908BD4FF4887103487F
:1006F000FFF7B8FF783D0020004800402838000888
:1007000008B50D484FF0A043036004234360022264
:10071000C26000230361436182610122C2610362FE
:100720004362C262036301F0F3F800B908BD4FF4FD
:1007300093710248FFF796FFB83D00202838000863
:1007400000B595B0002101912B4B1A6C42F08052FC
:100750001A641B6C03F080530193019B0291274B99
:100760001A6842F440421A601B6803F44043029343
:10077000029B012308934FF4A023099302230E93B5
:100780004FF480020F9204221092A8221192129329
:100790000723139308A801F095FA20BB0F230393B6
:1007A00002230493002305934FF4A05306934FF4C0
:1007B00080530793052103A801F040FDB8B901F06B
:1007C00047FE0F4BA3FB0030800902F0B1F8042074
:1007D00002F0C4F800220F214FF0FF3002F04CF875
:1007E00015B05DF804FBC6210648FFF73BFFD42196
:1007F0000448FFF737FF00BF003802400070004098
:10080000D34D62102838000800B587B002F0C4F854
:10081000FFF796FFFFF76CFEFFF726FFFFF752FF8B
:10082000FFF76EFF01AC074D0FCD0FC42B6823609F
:10083000002101A802F069FF034B186002F060FF7D
:10084000FEE700BF14380008743D00207047704771
:10085000FEE7FEE7FEE7FEE7704708B502F078FF27
:1008600008BD000008B5024800F050FC08BD00BFFC
:10087000F041002010B582B000240094214B5A6C46
:1008800042F480425A645A6C02F480420092009A08
:1008900001941A6C42F080521A641B6C03F080536E
:1008A0000193019B032001F0C9FF224621466FF00E
:1008B0000B0001F0E1FF224621466FF00A0001F033
:1008C000DBFF224621466FF0090001F0D5FF2246EA
:1008D00021466FF0040001F0CFFF224621466FF061
:1008E000030001F0C9FF22460F216FF0010001F063
:1008F000C3FF22460F214FF0FF3001F0BDFF02B0D1
:1009000010BD00BF0038024002682B4B9A4200D055
:100910007047F0B589B000240094A3F590431A6B9A
:1009200042F000721A631A6B02F000720092009A91
:1009300001941A6B42F080621A631A6B02F08062B3
:100940000192019A02941A6B42F000621A631B6BC7
:1009500003F000630293029B322303930227049760
:100960000594032606960B25079503A9134801F065
:10097000B3FD86230393049705940696079503A970
:100980000F4801F0A9FD4FF4005303930497059419
:100990000696079503A90B4801F09EFD4FF42053DE
:1009A0000393049705940696079503A9064801F05A
:1009B00093FD09B0F0BD00BF008002400008024076
:1009C0000000024000040240001802400268124B7E
:1009D0009A4200D0704700B587B0002300930F4BB8
:1009E0001A6C42F480221A641B6C03F48023009377
:1009F000009B4FF44073019302230293012303935E
:100A0000032304930723059301A9054801F064FD1E
:100A100007B05DF804FB00BF00480040003802400A
:100A2000000C02400368B3F1A04F00D0704730B50E
:100A300087B04FF4E85301930223029300240394F8
:100A4000032304930A2305930F4D01A9284601F0BF
:100A500043FD4FF4007301930294039401A92846C7
:100A600001F03AFD094B5A6B42F080025A63009440
:100A70005A6C42F480425A645B6C03F480430093E6
:100A8000009B07B030BD00BF0000024000380240AC
:100A900010B588B000220146192001F0EDFE1920A2
:100AA00001F030FF00240194144B5A6C42F0010213
:100AB0005A645B6C03F001030193019B02A903A834
:100AC00001F0ECFC01F0DAFC43000D48A0FB03232D
:100AD0009B0C013B0B480C4A026040F2E732C260BB
:100AE00043600461846000F02FFC10B1012008B065
:100AF00010BD044800F0B8FAF9E700BF0038024022
:100B000083DE1B43F04100200000014038B514464D
:100B10000D4651B1082908D0102906D0182904D053
:100B200040F24F710A48FFF791FE6279237943EA58
:100B30000223084AAB50E278A3781B0443EA02631D
:100B4000627843EA022322781343034AAB5038BD4C
:100B500040380008408002404480024070B59EB09A
:100B6000044629B14FF40063C3604FF480438360AF
:100B7000E369002B6AD14FF48063079321680B6807
:100B8000394A1A40A368E06803430798034343F4D3
:100B9000007313430B6023681D68012001F028FFD8
:100BA00023681D60236840225A6023685D68012025
:100BB00001F01EFF23685D60236800259D602368A7
:100BC000DD602268936923F0BE031B041B0C43F015
:100BD0008003936123689E69012001F009FF236867
:100BE0009E612368DD612368DD69012001F000FF5B
:100BF0002368DD61226841F2180551591B4B0B40F7
:100C000043F0087343F00403535123685E590120F5
:100C100001F0EEFE23685E51236803F58053144A09
:100C20001A60236803F580531D68012001F0E0FE7F
:100C3000236803F580531D60A369012B09D0626905
:100C400000212046FFF762FF1EB070BD002307930E
:100C500094E7216841F21C028B5843F4803343F03F
:100C600040038B50EBE700BF0F8120FF233FDEF8EE
:100C70008020C102F8B506460D461746038A202B90
:100C800025D896F84430DBB2822B37D0822386F801
:100C900044303268136903F01C03348AE402A4B2BE
:100CA0002343AC0104F4F8641C4344F001041461D0
:100CB00001F098FE054614F0010F16D001F092FEE7
:100CC000401BB0F5803F08D233681C69F3E74FF44E
:100CD00085610B48FFF7BAFDD3E7012386F844305E
:100CE000002386F84530032007E033685B699BB238
:100CF0003B60012386F844300020F8BD0220FCE769
:100D000040380008F8B506460D461746038A202BE2
:100D100028D896F84430DBB2422B36D0422386F8EE
:100D200044303268136903F01C03348AE402A4B22D
:100D30002343AC0104F4F8641C4344F00304BFB241
:100D4000576133681C6101F04DFE054614F0010F38
:100D500016D001F047FE401BB0F5803F08D2336843
:100D60001C69F3E74FF48E610948FFF76FFDD0E788
:100D7000012386F84430002386F84530032003E041
:100D8000012386F844300020F8BD0220FCE700BFB4
:100D90004038000870B582B000230193002800F0AD
:100DA000498104464368012B43D8A369012B45D8E8
:100DB000E369012B47D8236A13B1B3F5000F47D17C
:100DC00094F84430002B48D0002300939A4B5A6C7F
:100DD00042F480425A645B6C03F480430093009BAE
:100DE000964B5A6822F400025A605A68216A0A43F4
:100DF0005A60236803F580531A6842F001021A60B2
:100E000001F0F0FD0546236803F58052126812F0E8
:100E1000010F28D001F0E6FD401BB0F5FA7FF2D9B2
:100E2000032584F84450002384F84530284602B056
:100E300070BDC0218248FFF709FDB6E7C121804897
:100E4000FFF704FDB4E7C2217D48FFF7FFFCB2E7DE
:100E5000C3217B48FFF7FAFCB2E784F8453020460F
:100E6000FFF752FDB0E71D6925F01C0501F0F0FA0F
:100E7000744B0344744A934239D845F008052368FB
:100E80001D614FF4004200212046FFF73BFF05465D
:100E9000002844D1FF2001F0ABFD6368002B46D150
:100EA000A3681BB1B3F5804F40F0B080E368B3F5A1
:100EB000006F02D0002B40F0AF80E268C2F3CF0297
:100EC000A368C3F34F031A4300212046FFF71AFF1C
:100ED000002840F0A78040F6FF7001F089FD002156
:100EE0002046FFF73BFE012384F844309EE7574B32
:100EF0000344574A934202D845F00C05BFE7554BCF
:100F00000344554A9342BAD9544B0344544A93423A
:100F100002D845F00405B2E745F01005AFE701211E
:100F20002046FFF71BFE012584F844507EE701F0C0
:100F300059FD064601AA01212046FFF79BFE01F05C
:100F400051FD801B41F28833984230D8019B13F049
:100F5000040FEFD04FF4805200212046FFF7D2FE5D
:100F600088BB01F03FFD064601AA01212046FFF79C
:100F700081FE01F037FD801B41F2883398422AD868
:100F8000019B13F0200FEFD001AA10212046FFF79C
:100F900071FE60BB019B13F0040F30D04FF4006270
:100FA000E26013F0020F2DD00023A36097E7012128
:100FB0002046FFF7D3FD012384F84430002384F852
:100FC0004530032532E701212046FFF7C7FD012503
:100FD00084F844502AE701212046FFF7BFFD012392
:100FE00084F84430002384F8453003251EE70121AE
:100FF0002046FFF7B3FD012584F8445016E7002290
:10100000E260CEE74FF48043A36068E74FF4CD7110
:101010000B48FFF71BFC49E740F29B110848FFF71C
:1010200015FC4AE701212046FFF798FD012584F8C9
:101030004450FBE60125F9E6003802400038014043
:101040004038000800D3CEFEBFE1E40040F1E9FDE6
:101050003F787D0100796CFCFF596202001F0AFA9B
:101060007FF0FA027047000010B504460368234A77
:10107000934237D0B3F1804F34D0A2F57C429342F3
:1010800030D002F5806293422CD002F58062934208
:1010900028D002F58062934224D002F58062934208
:1010A00020D002F5704293421CD002F57052934258
:1010B00018D002F58062934214D002F58062934208
:1010C00010D0A2F5983293420CD002F58062934280
:1010D00008D002F58062934204D04FF4B171084801
:1010E000FFF7B4FB2268D36843F00103D3602268A2
:1010F000136843F001031360002010BD000001409D
:1011000078380008704770477047704710B504463C
:1011100003681A6912F0020F11D0DA6812F0020F98
:101120000DD06FF002021A610123037603689B69F8
:1011300013F0030F70D0FFF7E6FF00232376236838
:101140001A6912F0040F12D0DA6812F0040F0ED0F0
:101150006FF004021A610223237623689B6913F45B
:10116000407F5FD02046FFF7CEFF00232376236821
:101170001A6912F0080F12D0DA6812F0080F0ED0B8
:101180006FF008021A61042323762368DB6913F0E9
:10119000030F4ED02046FFF7B6FF002323762368C7
:1011A0001A6912F0100F12D0DA6812F0100F0ED078
:1011B0006FF010021A61082323762368DB6913F4A9
:1011C000407F3DD02046FFF79EFF00232376236813
:1011D0001A6912F0010F03D0DA6812F0010F36D14C
:1011E00023681A6912F0800F03D0DA6812F0800FBA
:1011F00034D123681A6912F0400F03D0DA6812F074
:10120000400F32D123681A6912F0200F03D0DA6838
:1012100012F0200F30D110BDFFF774FF2046FFF70A
:1012200073FF8AE72046FFF76DFF2046FFF76CFF4C
:101230009BE72046FFF766FF2046FFF765FFACE718
:101240002046FFF75FFF2046FFF75EFFBDE76FF028
:1012500001021A612046FFF7F9F9C1E76FF0800239
:101260001A61204600F0E7F8C3E76FF040021A6108
:101270002046FFF74AFFC5E76FF020021A612046BB
:1012800000F0D8F8C7E7000003682E4A904212D059
:10129000B0F1804F0FD0A2F57C4290420BD002F506
:1012A0008062904207D002F58062904203D002F53E
:1012B0007842904203D123F070034A681343214AD5
:1012C00090422AD0B0F1804F27D0A2F57C429042C4
:1012D00023D002F5806290421FD002F580629042D6
:1012E0001BD002F57842904217D002F5705290421E
:1012F00013D002F5806290420FD002F580629042D6
:101300000BD0A2F59832904207D002F5806290424D
:1013100003D002F58062904203D123F44073CA687F
:10132000134303608B68C3620B688362054B98426A
:1013300003D003F58063984201D10B690363012355
:10134000436170470000014000286DD010B504468D
:101350000368364A934236D0B3F1804F33D0A2F5BA
:101360007C4293422FD002F5806293422BD002F54B
:101370008062934227D002F58062934223D002F527
:10138000806293421FD002F5704293421BD002F557
:101390007052934217D002F58062934213D002F547
:1013A000806293420FD0A2F5983293420BD002F59F
:1013B0008062934207D002F58062934203D0D72126
:1013C0001B48FFF743FAA3683BB1102B05D0202B35
:1013D00003D0402B01D0602B16D123692BB1B3F57C
:1013E000807F02D0B3F5007F13D194F83930ABB1D0
:1013F000022384F83930211D2068FFF745FF0123BF
:1014000084F83930002010BDD8210948FFF71EFAB2
:10141000E3E7D9210648FFF719FAE6E784F8383000
:101420002046FFF71FFEE3E7012070470000014060
:1014300078380008704770472DE9F8430446426841
:10144000B44B9A4200F29C80E3681BB1B3F5005F95
:1014500040F09C80236933B1B3F5806F03D0B3F5BE
:10146000C06F40F0998063694FF6F372134200D168
:1014700023B940F68811A848FFF7E8F921680A69FE
:1014800022F44052E36813430B612168CA6822F4D6
:10149000164222F00C02A3682069034360690343EB
:1014A000E06903431343CB6021684A6922F4407228
:1014B000A36913434B61E369B3F5004F72D023680E
:1014C000964A934200F02E8102F58062934200F02A
:1014D000298100F0C3FF00EB800000EB800065680D
:1014E000AD00B0FBF5F58E4FA7FB05356D092E015C
:1014F00000F0B4FF00EB800000EB80006568AD00F9
:10150000B0FBF5F900F0AAFF00EB800000EB8000D3
:101510006568AD00B0FBF5F5A7FB05356D094FF02B
:10152000640808FB15952D013235A7FB05356D09BB
:1015300005F0F005354400F091FF00EB800000EB72
:1015400080006668B600B0FBF6F600F087FF00EB9F
:10155000800000EB800063689B00B0FBF3F0A7FB0A
:101560000030400908FB10684FEA081808F13208FB
:10157000A7FB0837C7F3431723682F449F6027E171
:1015800040F685116448FFF761F95DE740F6861182
:101590006148FFF75BF95DE740F687115E48FFF7AA
:1015A00055F960E723685D4A93425BD002F580629B
:1015B000934257D000F052FF00EB800000EB800018
:1015C00065686D00B0FBF5F5554FA7FB05356D0956
:1015D0002E0100F043FF00EB800000EB8000656807
:1015E0006D00B0FBF5F900F039FF00EB800000EB77
:1015F000800065686D00B0FBF5F5A7FB05356D094A
:101600004FF0640808FB1595ED003235A7FB053552
:101610006D096D0005F4F875354400F01FFF00EB0F
:10162000800000EB800066687600B0FBF6F600F004
:1016300015FF00EB800000EB800063685B00B0FBEF
:10164000F3F3A7FB03235B0908FB13684FEAC80801
:1016500008F13208A7FB0837C7F3421723682F4465
:101660009F60B5E000F00AFF00EB800000EB800017
:1016700065686D00B0FBF5F5294FA7FB05356D09D1
:101680002E0100F0FBFE00EB800000EB800065689F
:101690006D00B0FBF5F900F0F1FE00EB800000EB0F
:1016A000800065686D00B0FBF5F5A7FB05356D0999
:1016B0004FF0640808FB1595ED003235A7FB0535A2
:1016C0006D096D0005F4F875354400F0D7FE00EBA8
:1016D000800000EB800066687600B0FBF6F600F054
:1016E000CDFE00EB800000EB800063685B00B0FB88
:1016F000F3F3A7FB03235B0908FB13684FEAC80851
:1017000008F13208A7FB0837C7F3421723682F44B4
:101710009F605DE0A037A000B038000800100140D5
:101720001F85EB5100F0AAFE00EB800000EB80006B
:101730006568AD00B0FBF5F5264FA7FB05356D09D3
:101740002E0100F09BFE00EB800000EB800065683E
:10175000AD00B0FBF5F900F091FE00EB800000EB6E
:1017600080006568AD00B0FBF5F5A7FB05356D0998
:101770004FF0640808FB15952D013235A7FB0535A0
:101780006D0905F0F005354400F078FE00EB8000AF
:1017900000EB80006668B600B0FBF6F600F06EFE67
:1017A00000EB800000EB800063689B00B0FBF3F06F
:1017B000A7FB0030400908FB10684FEA081808F141
:1017C0003208A7FB0837C7F3431723682F449F60ED
:1017D000BDE8F8831F85EB51002800F0938010B519
:1017E00004468369002B55D00368474A934210D0C2
:1017F000A2F54C4293420CD002F58062934208D08D
:1018000002F54C42934204D04FF480713F48FFF7F9
:101810001DF8A36943B1B3F5807F05D0B3F5007F10
:1018200002D0B3F5407F2FD1A36813B1B3F5805F29
:1018300056D1E36913B1B3F5004F57D194F839305D
:10184000002B59D0242384F839302268D36823F43C
:101850000053D3602046FFF7EFFD2268136923F49D
:10186000904313612268536923F02A03536122686D
:10187000D36843F40053D3600020E063202384F84E
:10188000393084F83A3010BD40F201111F48FEF79C
:10189000DDFFC9E703681C4A9342C5D0A2F54C425C
:1018A0009342C1D002F580629342BDD002F58062BE
:1018B0009342B9D002F580629342B5D002F544421A
:1018C0009342B1D0A2F51C429342ADD002F58062A2
:1018D0009342A9D040F205110C48FEF7B7FFA3E7E9
:1018E00040F207110948FEF7B1FFA2E74FF48471F7
:1018F0000648FEF7ABFFA1E784F838302046FFF733
:1019000065F89FE70120704700100140B0380008DB
:10191000002877D0F0B58BB004460368B3F1A04F30
:1019200006D0394A934203D094213848FEF78EFFFF
:10193000032384F8B9332046FFF774F8206800F0D9
:10194000A5F8254655F8107B6E460FCD0FC60FCD76
:101950000FC695E8030086E80300231D0ECB38462A
:1019600000F056F80021206800F096F8002210E000
:10197000D100891A8B002344012183F8391083F8A0
:101980003820DA87002183F83B1019645964D96440
:1019900001320E2AECD9002218E0D100891A8B00FE
:1019A0002344002183F8F91183F8F821DA8783F8BA
:1019B000FB11C3F80012C3F80412C3F80C12236819
:1019C00002F1400003EB8003596001320E2AE4D992
:1019D000254655F8107B6E460FCD0FC60FCD0FC6AE
:1019E00095E8030086E80300231D0ECB384600F07F
:1019F00069F8012384F8B933206800F038F9002031
:101A00000BB0F0BD0120704700000440E83800082A
:101A100084B010B5044603A880E80E00089B012B93
:101A200020D1A36B23F48033A363E36823F48403FE
:101A300023F04003E360E36823F44013E3600F9B6B
:101A4000012B0AD0204600F01FF9069B012B14D071
:101A50000020BDE8104004B07047E36843F48013F1
:101A6000E360EFE7E36843F04003E360204600F003
:101A70000BF94FF48033A363E7E7A36843F0060351
:101A8000A360A36843F02003A360E1E7836823F029
:101A9000010383600020704708B5C36823F0C0438A
:101AA000C360012909D019B9C36843F08043C360FA
:101AB000322000F09DFF002008BDC36843F00053B2
:101AC000C360F5E784B0F8B5044607A880E80E00C7
:101AD000119FBFB9A36B43F40013A36325460023F2
:101AE000C4F8003E04F50066D4F80038C4F80038A5
:101AF0000C9B012B10D1099B4BB90021204600F013
:101B0000AFF80DE0A36B43F40023A363E6E70121E4
:101B1000204600F0A5F803E00321204600F0A0F8DD
:101B20001021204600F076F8204600F087F80023C8
:101B3000336173614FF0FF32B261F36108E04FF03F
:101B40009040C2F8000900220A61FF228A60013336
:101B5000079999420BD905EB431202F51061D2F8AF
:101B600000090028EBDB0020C2F80009EBE70023A6
:101B700008E04FF0904CC2F800CB00220261FF2237
:101B80008260013399420DD905EB431202F53060B2
:101B9000D2F800CBBCF1000FEBDB4FF0000CC2F829
:101BA00000CBEAE7336923F4807333610A9B012B8E
:101BB0001AD00022A2616FF0804262611BB9A36952
:101BC00043F01003A361A269104B1343A3610D9B63
:101BD0001BB1A36943F00803A361012F0ED00020BD
:101BE000BDE8F84004B07047094A3263326B42F4F2
:101BF000803242F003023263326BDAE7A36943F0CA
:101C0000804343F00403A361E9E700BF00383C8050
:101C100000018000890141F02001016100230133AE
:101C2000054A934205D8026912F0200FF7D100202F
:101C300070470320704700BF400D0300102303616D
:101C400000230133054A934205D8026912F0100FB0
:101C5000F7D1002070470320704700BF400D0300FC
:101C6000D0F800381943C0F800180020704708B5B4
:101C7000D0F8043843F00203C0F80438032000F021
:101C8000B7FE002008BD0000002301330C4A934238
:101C900011D80269002AF8DA036943F001030361ED
:101CA00000230133064A934207D8026912F0010F5C
:101CB000F7D100207047032070470320704700BF12
:101CC000400D0300002800F03C8270B582B004464D
:101CD00003680F2B39D8236813F0010F4DD06368C8
:101CE0002BB1B3F5803F02D0B3F5A02F32D1A54B75
:101CF0009B6803F00C03042B36D0A24B9B6803F0C7
:101D00000C03082B2BD06368B3F5803F5FD0B3F58D
:101D1000A02F62D09B4B1A6822F480321A601A6896
:101D200022F480221A606368002B60D000F05AFE13
:101D30000546944B1B6813F4003F1ED100F052FE81
:101D4000401B6428F5D9032000E2F8218E48FEF7F5
:101D50007DFDC0E7FD218C48FEF778FDC7E7894B84
:101D60005B6813F4800FCED0864B1B6813F4003FE2
:101D700003D06368002B00F0E681236813F0020FA4
:101D800067D0E368012B41D823691F2B44D87D4BD2
:101D90009B6813F00C0F4AD07A4B9B6803F00C033E
:101DA000082B3FD0E368002B77D0784B01221A60D4
:101DB00000F018FE0546734B1B6813F0020F63D149
:101DC00000F010FE401B0228F5D90320BEE16D4A49
:101DD000136843F480331360A5E76A4B1A6842F432
:101DE00080221A601A6842F480321A609BE700F081
:101DF000F9FD0546634B1B6813F4003FBDD000F0AE
:101E0000F1FD401B6428F5D903209FE140F22F111A
:101E10005D48FEF71BFDB7E74FF498715A48FEF78F
:101E200015FDB4E7574B5B6813F4800FBAD1554BDF
:101E30001B6813F0020F04D0E368012B01D00120CE
:101E400084E1504A136823F0F803216943EAC1038F
:101E50001360236813F0080F49D06369012B2ED853
:101E6000636993B34A4B01221A6000F0BBFD05463B
:101E7000444B5B6F13F0020F39D100F0B3FD401BF0
:101E80000228F5D9032061E13E4A136823F0F803E4
:101E9000216943EAC1031360DBE73C4B00221A606F
:101EA00000F0A0FD0546374B1B6813F0020FD0D0A1
:101EB00000F098FD401B0228F5D9032046E14FF4BD
:101EC000B8713148FEF7C2FCCAE7314B00221A60F4
:101ED00000F088FD05462B4B5B6F13F0020F06D018
:101EE00000F080FD401B0228F5D903202EE1236875
:101EF00013F0040F00F08780A368012B01D9052B94
:101F000038D1204B1B6C13F0805F39D10023019333
:101F10001C4B1A6C42F080521A641B6C03F0805305
:101F20000193019B01251B4B1B6813F4807F33D069
:101F3000A368012B44D0052B48D0124B1A6F22F016
:101F400001021A671A6F22F004021A67A368002BB5
:101F500046D000F047FD06460A4B1B6F13F0020FF8
:101F60004FD100F03FFD801B41F288339842F3D9F6
:101F70000320EBE04FF4CE710348FEF767FCC0E7A7
:101F80000025D0E700380240203900080000474211
:101F9000800E4742007000406E4A136843F480731D
:101FA000136000F01FFD06466A4B1B6813F4807F28
:101FB000BED100F017FD801B0228F5D90320C5E033
:101FC000654A136F43F001031367BFE7624B1A6F53
:101FD00042F004021A671A6F42F001021A67B5E76D
:101FE00000F000FD06465C4B1B6F13F0020F08D09B
:101FF00000F0F8FC801B41F288339842F3D90320AB
:10200000A4E0002D3BD1A369022B3ED8A369002B8D
:1020100000F09B80504A926802F00C02082A00F0FF
:102020009780022B79D1E36913B1B3F5800F32D1D8
:10203000236A3F2B35D8636A323BB3F5BF7F36D86E
:10204000A36A022B05D0042B03D0062B01D0082B4A
:1020500033D1E36A023B0D2B35D8404B00221A6086
:1020600000F0C0FC05463C4B1B6813F0007F30D0ED
:1020700000F0B8FC401B0228F5D9032066E0364A80
:10208000136C23F080531364BDE740F2DF11344832
:10209000FEF7DCFBBAE74FF4F4713148FEF7D6FBEC
:1020A000C6E740F2E9112E48FEF7D0FBC3E74FF434
:1020B000F5712B48FEF7CAFBC2E740F2EB11284846
:1020C000FEF7C4FBC5E74FF4F6712548FEF7BEFBEB
:1020D000C3E7E369226A1343626A43EA8213A26A8E
:1020E0005208013A43EA0243E26A43EA02631A4AA7
:1020F00053601A4B01221A6000F074FC0446164B20
:102100001B6813F0007F06D100F06CFC001B022856
:10211000F5D903201AE0002018E0104B00221A60C5
:1021200000F060FC04460C4B1B6813F0007F06D0E7
:1021300000F058FC001B0228F5D9032006E000201F
:1021400004E001207047012000E0002002B070BDD3
:102150000120FBE700700040003802406000474269
:1021600020390008324B9B6803F00C03042B5CD031
:10217000082B01D02F4870472DE9F04B2C4B5A68A3
:1021800002F03F025B6813F4800F2BD0284B5B6892
:10219000C3F388131E4600275C010025E41A65EB93
:1021A0000705A90141EA9461A001001B61EB05014B
:1021B000CB0043EA5073C400A01943EB07014B0264
:1021C00043EAD0534402204619460023FEF710F894
:1021D000174B5B68C3F3014301335B00B0FBF3F0C3
:1021E000BDE8F08B124B5B68C3F388131E460027D3
:1021F0005C010025E41A65EB0705A90141EA946139
:10220000A001001B61EB0501CB0043EA5073C40041
:10221000A01943EB07018B0243EA90538402204646
:1022200019460023FDF7E4FFD2E70348704700BFDB
:10223000003802400024F40000127A00002800F068
:10224000F98070B504460D460368013B0E2B11D88A
:102250000F2D15D8794B1B6803F00F03AB4215D235
:10226000EBB2764A1370136803F00F03AB420DD044
:10227000012070BD4FF414717148FEF7E7FAE7E7EB
:1022800040F251216E48FEF7E1FAE3E7236813F0CC
:10229000020F29D013F0040F04D06A4A936843F464
:1022A000E0539360236813F0080F04D0654A9368E5
:1022B00043F460439360A3687BB1802B0DD0902BD7
:1022C0000BD0A02B09D0B02B07D0C02B05D0D02B22
:1022D00003D0E02B01D0F02B33D15A4A936823F07E
:1022E000F003A1680B439360236813F0010F42D001
:1022F0006368032B2BD86368012B2ED09A1E012A0A
:1023000032D9504A126812F0020F00F095804D4900
:102310008A6822F0030213438B6000F063FB0646D9
:10232000484B9B6803F00C036268B3EB820F22D02A
:1023300000F058FB801B41F288339842F0D903200B
:1023400097E74FF41D713E48FEF780FAC5E740F26B
:102350007B213B48FEF77AFACDE73A4A126812F43D
:10236000003FD4D1012084E7364A126812F0007F82
:10237000CDD101207DE7314B1B6803F00F03AB4249
:1023800009D9EAB22D4B1A701B6803F00F03AB4258
:1023900001D001206DE7236813F0040F14D0E36827
:1023A0005BB1B3F5805F08D0B3F5A05F05D0B3F59E
:1023B000C05F02D0B3F5E05F30D1224A936823F4C6
:1023C000E053E1680B439360236813F0080F15D0C6
:1023D00023695BB1B3F5805F08D0B3F5A05F05D08A
:1023E000B3F5C05F02D0B3F5E05F1DD1154A936825
:1023F00023F46043216943EAC1039360FFF7B2FE0F
:10240000104B9B68C3F303130F4AD35CD8400F4BA8
:1024100018600020FEF73CFB00202AE740F2B921BB
:102420000748FEF713FAC8E74FF430710448FEF787
:102430000DFADBE70120704701201AE7003C02405B
:102440002039000800380240C83900080400002084
:10245000014B1868704700BF0400002008B5FFF763
:10246000F7FF044B9B68C3F38223034AD35CD84035
:1024700008BD00BF00380240D839000808B5FFF792
:10248000E7FF044B9B68C3F34233034AD35CD84055
:1024900008BD00BF00380240D83900080F23036090
:1024A0000B4B9A6802F0030242609A6802F0F00255
:1024B00082609A6802F4E052C2609B68DB0803F411
:1024C000E0530361034B1B6803F00F030B6070477D
:1024D00000380240003C02402DE9F04782B08046BF
:1024E0000E46BD4B98422BD003F58063984227D00F
:1024F00003F58063984223D003F5806398421FD090
:1025000003F5806398421BD003F58063984217D08F
:1025100003F58063984213D003F5806398420FD08F
:1025200003F5806398420BD003F58063984207D08F
:1025300003F58063984203D0C321A848FEF786F9CB
:1025400033689AB212B11B0C1B041BB1C421A348FF
:10255000FEF77CF97368012B1ED9112B1CD0022BBE
:102560001AD0122B18D09E4A934215D002F5801231
:10257000934211D002F5801293420DD0A2F5F812C9
:10258000934209D002F58012934205D002F58012E1
:10259000934201D0032B04D1B368022B06D8002448
:1025A0004AE0C5218D48FEF751F9F5E7C6218B4871
:1025B000FEF74CF9F3E7D7218848FEF747F969E0C1
:1025C000EA218648FEF742F994E0092300E000235F
:1025D0008B4003430232834941F82230824B1A6810
:1025E000FB4303EA0201706810F4803F01D047EA20
:1025F00002017D4A1160526803EA0201706810F41A
:10260000003F01D047EA0201774A5160926803EA2D
:102610000201706810F4801F01D047EA0201724A7B
:102620009160D2681340716811F4001F01D047EA2D
:1026300002036D4AD36001340F2C00F2DF800125C4
:10264000A54037682F40BD42F5D17368022B01D0F9
:10265000122B2FD13369EBB1092B1BD0012B19D0D1
:10266000022B17D0032B15D0042B13D0052B11D020
:10267000062B0FD0072B0DD0082B0BD00A2B09D01F
:102680000B2B07D00C2B05D00D2B03D00F2B01D01B
:102690000E2B90D1E208083258F8220004F007030C
:1026A00099000F238B4020EA030033698B400343DA
:1026B00048F82230D8F800204FEA440A4FF00309C6
:1026C00009FA0AF96FEA090909EA0202736803F0D4
:1026D000030303FA0AF31343C8F8003073685A1E61
:1026E000012A03D9112B01D0122B18D1F368032B27
:1026F0003FF666AFD8F8082009EA0202F36803FA49
:102700000AF31343C8F80830D8F8042022EA050277
:102710007368C3F30015A5401543C8F80450D8F8F2
:102720000C3009EA0309B36803FA0AF343EA090320
:10273000C8F80C30736813F0805F3FF47CAF00235F
:1027400001932A4B5A6C42F480425A645B6C03F446
:1027500080430193019BA208911C224B53F8210056
:1027600004F0030399000F238B4020EA03001A4B67
:1027700098453FF42CAF03F58063984522D003F5CC
:102780008063984520D003F5806398451ED003F5FB
:10279000806398451CD003F5806398451AD003F5F3
:1027A0008063984524D003F58063984522D003F5D3
:1027B0008063984520D003F5806398453FF405AFCA
:1027C0000A2305E7012303E7022301E70323FFE6CA
:1027D0000423FDE60523FBE600000240583900080B
:1027E0000000111000380140003C01400038024058
:1027F0000623EDE60723EBE60823E9E602B0BDE891
:10280000F08700BF70B5064615460C4629B1012D6C
:1028100009D875B92404B46170BD40F2AF110648FF
:10282000FEF714F8F3E74FF4D8710348FEF70EF8FB
:10283000EFE7B461F0E700BF5839000810B504466F
:10284000C31E042B0FD80A4AD36823F4E0631B0489
:102850001B0C240204F4E064234343F0BF6343F4FD
:102860000033D36010BDA2210248FDF7EFFFEAE775
:1028700000ED00E09039000870B505460C4616469C
:102880000F2A25D80F2C28D81B4BDB68C3F3022353
:10289000C3F10702042A28BF0422191D062921D9E1
:1028A000033B4FF0FF3101FA02F224EA02049C409C
:1028B00001FA03F326EA03063443002D14DB240156
:1028C000E4B205F1604505F5614585F8004370BD4A
:1028D000BA210A48FDF7BAFFD4E7BB210748FDF744
:1028E000B5FFD1E70023DCE705F00F052401E4B2D2
:1028F000034B5C55EBE700BF00ED00E090390008AA
:1029000014ED00E010B5041E08DB04F01F0264099A
:1029100001239340044A42F8243010BDCE210348DD
:10292000FDF794FFF1E700BF00E100E090390008F7
:102930000138B0F1807F0AD2064B5860064AF02178
:1029400082F823100020986007221A607047012047
:10295000704700BF10E000E000ED00E010B5044655
:10296000042800D038B9042C0BD0094A136823F08E
:102970000403136010BD40F2D9110648FDF766FF4D
:10298000F1E7034A136843F004031360F2E700BF62
:1029900010E000E09039000808B50B4B1A6842F4CB
:1029A00000721A601A6842F480621A601A6842F46F
:1029B00080721A600320FFF741FF0020FEF768F8DD
:1029C000FDF758FF002008BD003C0240034A116893
:1029D000034B1B780B441360704700BF2C42002050
:1029E00000000020014B1868704700BF2C420020F7
:1029F00038B50446FFF7F6FF0546B4F1FF3F02D0B5
:102A0000044B1B781C44FFF7EDFF401BA042FAD398
:102A100038BD00BF000000200F49D1F8883043F4D2
:102A20007003C1F888300D4B1A6842F001021A6039
:102A3000002098601A6822F0847222F480321A60B2
:102A4000074A5A601A6822F480221A60D8604FF050
:102A500000638B60704700BF00ED00E0003802406B
:102A600010300024124A12F0070F1ED0D11D21F0A1
:102A70000701C1F5705313440A460E480260002155
:102A800041601344083B23F007030B48036059607F
:102A90001960991A51601360084B1960084B19604E
:102AA000084B4FF000421A6070474FF47053E4E750
:102AB0002C000020383C002028000020343C00205E
:102AC000303C00202C3C002010B4134B1A6882428A
:102AD0001BD359685C18844203D140680144596093
:102AE000184641684418A24213D10C4C2468A242F3
:102AF0000DD05268114441601A6812680260984211
:102B000000D018605DF8044B70471346DEE70460A0
:102B1000F5E70260F3E700BF383C00202800002002
:102B200070B5044600F014FC3A4B1B68BBB13A4B3D
:102B30001B681C4263D1ACB1083414F0070F11D0EC
:102B400024F00704083404F007035BB14FF050038E
:102B500083F31188BFF36F8FBFF34F8FFEE7FFF74B
:102B600081FFE4E7002C4CD02C4B1B68A3424AD3D6
:102B70002B4B1D6801E02B4615466A68A24202D223
:102B80002A68002AF7D1234A1268AA423DD01E685B
:102B900008362A681A606B681B1B102B10D928197D
:102BA00010F0070F08D04FF0500383F31188BFF3E4
:102BB0006F8FBFF34F8FFEE743606C60FFF784FFBA
:102BC0006A6816490B689B1A0B60164909688B42A4
:102BD00001D214490B60104B1B6813436B60002338
:102BE0002B6000F049FC16F0070F10D04FF0500397
:102BF00083F31188BFF36F8FBFF34F8FFEE700267B
:102C0000EFE70026EDE70026EBE70026E9E7304690
:102C100070BD00BF280000202C3C0020303C00206C
:102C2000383C0020343C002080B338B50446A0F185
:102C3000080550F8042C164909680A4208D14FF0DB
:102C4000500383F31188BFF36F8FBFF34F8FFEE7FD
:102C500050F8080C40B14FF0500383F31188BFF3D4
:102C60006F8FBFF34F8FFEE722EA010244F8042C76
:102C700000F06EFB54F8041C064A13680B44136002
:102C80002846FFF721FF00F0F7FB38BD704700BF73
:102C90002C3C0020303C00200B4B1B68B3F1FF3F65
:102CA00008D04FF0500383F31188BFF36F8FBFF349
:102CB0004F8FFEE74FF0500383F31188BFF36F8F00
:102CC000BFF34F8FFEE700BF0800002006480068F2
:102CD000006880F3088862B661B6BFF34F8FBFF318
:102CE0006F8F00DF00BF000008ED00E0DFF80C0090
:102CF000016841F4700101607047000088ED00E058
:102D00004FF0807340F8043C21F0010140F8081CAA
:102D1000054B40F80C3C40F8202C6FF0020340F8C3
:102D2000243C4438704700BF992C00080000000084
:102D3000074B19680868B0E8F04F80F30988BFF3C3
:102D40006F8F4FF0000080F311887047AFF3008061
:102D5000483C00204FF0500383F31188BFF36F8F7E
:102D6000BFF34F8F0A4A136801331360012B00D061
:102D70007047084B1B6813F0FF0FF9D04FF050035A
:102D800083F31188BFF36F8FBFF34F8FFEE700BF50
:102D90000800002004ED00E0094B1B6843B94FF028
:102DA000500383F31188BFF36F8FBFF34F8FFEE79C
:102DB000013B034A13600BB983F31188704700BFCE
:102DC00008000020000000000000000000000000DB
:102DD000EFF30980BFF36F8F154B1A681EF0100FC9
:102DE00008BF20ED108A20E9F04F10604DF8043D37
:102DF0004FF0500080F31188BFF34F8FBFF36F8FF8
:102E000000F01CFC4FF0000080F3118808BC19682A
:102E10000868B0E8F04F1EF0100F08BFB0EC108A41
:102E200080F30988BFF36F8F704700BFAFF3008056
:102E3000483C002008B54FF0500383F31188BFF3DE
:102E40006F8FBFF34F8F00F08BFA18B1034B4FF029
:102E500080521A60002383F3118808BD04ED00E05E
:102E6000064B1B68064AA2FB03239B09013B054A4C
:102E70001360054B07221A60704700BF0400002052
:102E8000D34D621014E000E010E000E0314B1A680E
:102E9000314B9A420DD02F4B1A68304B9A4211D1C8
:102EA0004FF0500383F31188BFF36F8FBFF34F8F41
:102EB000FEE74FF0500383F31188BFF36F8FBFF32A
:102EC0004F8FFEE700B583B0254B1A78D2B201923E
:102ED000FF221A701B78DBB28DF803309DF80330A7
:102EE00003F050031F4A13701F4B07221A609DF80E
:102EF000033013F0800F0AD01B4A1368013B1360A4
:102F00009DF803305B00DBB28DF80330EFE7164A23
:102F100013681B0203F4E0631360019BDBB2104AE9
:102F20001370124B1A6842F470021A601A6842F069
:102F300070421A60FFF794FF0D4B00221A60FFF7F2
:102F4000D5FE0C4A136843F040431360FFF7BEFE02
:102F5000FFF7A2FE00ED00E071C20F4170C20F4109
:102F600000E400E0403C0020443C002020ED00E074
:102F70000800002034EF00E000F1080343604FF048
:102F8000FF328260C3600361002303607047002347
:102F90000361704743684B609A688A609A68516021
:102FA00099600861036801330360704730B40D68AD
:102FB000B5F1FF3F02D000F1080202E0026904E02F
:102FC0001A4653681C68AC42FAD953684B60996042
:102FD0008A605160086103680133036030BC704748
:102FE00003694268816891608268416851605A68EB
:102FF000824205D0002202611868013818607047CB
:1030000082685A60F6E70000084B1B681B683BB1FA
:10301000064B1B68DB68DB685A68054B1A60704713
:10302000034B4FF0FF321A60704700BF4C3C00204A
:10303000243D002010B50446006BFFF7F5FD204647
:10304000FFF7F2FD10BD2DE9F04780469946089D37
:10305000099F0A9C266B02F18042013A06EB820628
:1030600026F0070600230F2B07D8C85CE21882F869
:103070003400CA5C0AB10133F5E7002384F8433019
:10308000062D00D90625E56265644FF0000AC4F8F4
:1030900048A0201DFFF77BFF04F11800FFF777FF22
:1030A0002461C5F10705A5616462C4F84CA084F8E9
:1030B00050A04A4641463046FFF722FE206007B145
:1030C0003C60BDE8F087000038B5002407E004EB61
:1030D000840293000E481844FFF74EFF0134062C7B
:1030E000F5D90C4D2846FFF747FF0B4C2046FFF75C
:1030F00043FF0A48FFF740FF0948FFF73DFF094833
:10310000FFF73AFF084B1D60084B1C6038BD00BF3D
:10311000543C0020F83C00200C3D00202C3D0020B9
:10312000583D0020443D00204C3C0020503C0020F5
:1031300010B50446FFF70EFE204A136801331360F2
:103140001F4B1B685BB11F4B1B686BB91C4B1B688B
:10315000DA6AE36A9A4207D8194B1C6004E0184BFC
:103160001C601368012B26D0174A136801331360C3
:10317000E36A01229A401549086802430A6003EB9A
:1031800083039A00211D12481044FFF703FFFFF745
:1031900003FE0C4B1B686BB1094B1B68DA6AE36AD0
:1031A0009A4207D20B4B4FF080521A60BFF34F8FF9
:1031B000BFF36F8F10BDFFF787FFD5E7E03C00201E
:1031C000483C0020403D0020F03C0020F43C002022
:1031D000543C002004ED00E070B504460E461D4B43
:1031E0001D681D4B18680430FFF7FAFE50B91A4BE2
:1031F0001B68DA6A012303FA02F218490B6823EA12
:1032000002030B60B4F1FF3F13D02C44124B1B6838
:103210005C60A54216D8124B18680F4B1968043130
:10322000FFF7C4FE0F4B1B68A34212D90D4B1C6065
:103230000FE0002EE9D0084B196804310A48FFF767
:10324000A9FE06E0094B1868034B19680431FFF723
:10325000ADFE70BD6C3D0020483C0020F43C0020D9
:103260004C3C0020243D0020443D0020503C0020E8
:103270002DE9F04385B007468846154699469000EB
:10328000FFF74EFCF8B106465420FFF749FC044610
:10329000A8B10663D4B10023039302940D9B01935C
:1032A0000C9B00934B462A4641463846FFF7CBFE1F
:1032B0002046FFF73DFF012005B0BDE8F083304612
:1032C000FFF7B2FCE6E74FF0FF30F5E74FF0FF30D5
:1032D000F2E7000000B583B0174B01930023009381
:1032E000802216491648FFF7C3FF012805D0B0F128
:1032F000FF3F17D003B05DF804FB4FF0500383F39A
:103300001188BFF36F8FBFF34F8F0E4B4FF0FF321B
:103310001A600D4B01221A600C4B00221A60FFF755
:10332000B5FDE7E74FF0500383F31188BFF36F8FCC
:10333000BFF34F8FFEE700BF203D0020E0390008BB
:1033400015360008243D0020403D00206C3D002043
:10335000024A136801331360704700BFEC3C002041
:10336000F8B53A4B1B68002B64D1394B1D68013509
:103370001D60C5B9374B1B681B6843B14FF0500344
:1033800083F31188BFF36F8FBFF34F8FFEE7314A8E
:103390001168314B186810601960304A13680133A6
:1033A0001360FFF731FE2E4B1B68AB4238D9002467
:1033B0002C4B1B68DB6A03EB83039A002A4B9B5858
:1033C000012B3CD901243AE00124224B1B681B68E5
:1033D00043B3204B1B68DB68DE6873689D4226D3CD
:1033E000371D3846FFF7FCFDB36A1BB106F1180024
:1033F000FFF7F6FDF36A01229A401C490868024370
:103400000A6003EB83039A00394617481044FFF71C
:10341000C1FDF26A134B1B68DB6A9A42D4D2D4E72F
:103420000024D2E70E4B4FF0FF321A60C0E70C4A7F
:103430001360BDE70E4A13680133136000240D4B7F
:103440001B6803B101242046F8BD00BFEC3C0020FE
:103450006C3D00204C3C0020503C0020283D0020CA
:10346000243D0020483C0020543C0020F43C002037
:10347000E83C0020703D002038B5334B1B6843B951
:103480004FF0500383F31188BFF36F8FBFF34F8F5B
:10349000FEE7FFF75FFC2C4B1A68013A1A601B68C5
:1034A000002B4DD1294B1B6823B90024FFF774FC76
:1034B000204638BD0024264B1B681BB3244BDB6819
:1034C000DC6804F11800FFF78BFD251D2846FFF787
:1034D00087FDE36A01229A401E49086802430A6098
:1034E00003EB83039A0029461B481044FFF752FD63
:1034F000E26A1A4B1B68DB6A9A42DCD3184B012242
:103500001A60D8E70CB1FFF77FFD164B1C6854B169
:10351000FFF726FF10B1124B01221A60013CF7D1D0
:10352000104B00221A600E4B1B685BB10E4B4FF024
:1035300080521A60BFF34F8FBFF36F8F0124B5E73E
:103540000024B3E70024B1E7EC3C0020E03C00207D
:103550002C3D0020F43C0020543C0020483C00203E
:10356000703D0020E83C002004ED00E010B5A8B15B
:1035700004460F4B1B6843B14FF0500383F311888F
:10358000BFF36F8FBFF34F8FFEE7FFF7E1FE002120
:103590002046FFF721FEFFF76FFF38B9054B4FF0CC
:1035A00080521A60BFF34F8FBFF36F8F10BD00BF03
:1035B000EC3C002004ED00E0134B1B6813B310B586
:1035C000FFF7C6FE114B1C68FFF756FF24B90E4BE0
:1035D0001B68002BF4D110BDFFF7BCFB0B4BDB6865
:1035E000DC68201DFFF7FCFC094A1368013B1360EF
:1035F000054A1368013B1360FFF7CEFB2046FFF737
:1036000019FDE4E7704700BFE43C0020583D00206E
:10361000E03C002008B5FFF7CFFF064B1B68012BED
:10362000F9D9054B4FF080521A60BFF34F8FBFF3AB
:103630006F8FF0E7543C002004ED00E0204B1B6846
:103640001BB1204B01221A6070471E4B00221A60EA
:103650001D4B1B68B3FA83F3DBB2C3F11F0303EB0B
:1036600083018A0019498A5842B94FF0500383F305
:103670001188BFF36F8FBFF34F8FFEE710B413486D
:103680009A00D418A10001444C6864684C601A4444
:1036900091000831084484420BD003EB83039A0065
:1036A0000A4B13445B68DA68094B1A605DF8044BF7
:1036B000704761680548142202FB03025160ECE781
:1036C000EC3C0020703D0020F43C0020543C0020E5
:1036D000483C0020054B1B6833B1054B1B680BB100
:1036E000002070470220704701207047403D0020B5
:1036F000EC3C0020842801D0033070470020704744
:1037000008B5FFF7E7FD002008BDF0B585B00F460E
:10371000446805680669B0F90800FFF7EBFF03ABE2
:10372000019300903B46B2B229462046FFF7A0FD28
:10373000012802D1039805B0F0BD0020FBE708B5D1
:10374000034600B901231846FFF710FF002008BD0B
:1037500008B5FFF7BFFF012801D0FFF76BFB08BDDD
:10376000DFF834D0002103E00C4B5B5843500431A8
:103770000B480C4B42189A42F6D30B4A02E0002346
:1037800042F8043B094B9A42F9D3FFF745F900F0A0
:1037900011F8FDF739F8704700000320F8390008E8
:1037A000000000200C0000200C000020304200200F
:1037B000FEE7000070B50D4E0D4CA41BA4100025B3
:1037C000A54209D10B4E0C4C00F018F8A41BA41014
:1037D0000025A54205D170BD56F825309847013522
:1037E000EEE756F8253098470135F2E7F039000842
:1037F000F0390008F0390008F4390008F8B500BFC6
:10380000F8BC08BC9E467047F8B500BFF8BC08BCC1
:043810009E46704719
:103814003438000819060008000000000000000009
:10382400800000005372632F6D61696E2E63000087
:1038340064656661756C745461736B004472697677
:103844006572732F53544D3332463478785F484150
:103854004C5F4472697665722F5372632F73746D73
:103864003332663478785F68616C5F6574682E63A0
:1038740000000000447269766572732F53544D330F
:1038840032463478785F48414C5F44726976657299
:103894002F5372632F73746D3332663478785F6894
:1038A400616C5F74696D2E63000000004472697678
:1038B4006572732F53544D3332463478785F4841E0
:1038C4004C5F4472697665722F5372632F73746D03
:1038D4003332663478785F68616C5F756172742E18
:1038E40063000000447269766572732F53544D333C
:1038F40032463478785F48414C5F44726976657229
:103904002F5372632F73746D3332663478785F6823
:10391400616C5F7063642E6300000000447269761A
:103924006572732F53544D3332463478785F48416F
:103934004C5F4472697665722F5372632F73746D92
:103944003332663478785F68616C5F7263632E63C8
:1039540000000000447269766572732F53544D332E
:1039640032463478785F48414C5F447269766572B8
:103974002F5372632F73746D3332663478785F68B3
:10398400616C5F6770696F2E630000004472697632
:103994006572732F53544D3332463478785F4841FF
:1039A4004C5F4472697665722F5372632F73746D22
:1039B4003332663478785F68616C5F636F72746504
:1039C400782E6300000000000000000001020304E0
:1039D40006070809000000000102030449444C459D
:0439E40000000000DF
:0839E80038C8FF7F0100000058
:0439F000D5010008F5
:0439F400B101000815
:0C39F800010000000024F400AAAAAAAA02
:040000050800376157
:00000001FF
